:08919F0033302E3320202000A4
:1080C2004105A100C100C102C1014105A200410553
:1080D200A6004105A7004105A8004105A9004105E8
:0280E200AA00F2
:0A917800E4F5847588107589022261
:0D4FF900E4F584759A4075F809759D302225
:10501B00E4F58475BCF8F5BA75E88075840275BC47
:05502B00F975E8802288
:0791B700E4F58475D10322E9
:1090A40075840F75AD0175A4CF75A50175A6777587
:0990B400A77F75E10375E3C022FA
:108DDE00E4FFFE75840F758A8353A1DFF58475B7A2
:108DEE00B075840F43A120438901758D01758F01E4
:108DFE00758E040FBF00010EEF640F4E70F54389A0
:098E0E0002E58930E4FB759702CE
:018E17002238
:0A91820075A88243E6F343E71222CA
:108EE400129178124FF912501B1291B71290A412DA
:108EF4008DDE129182AF84E4F58475D4808F8490E2
:0A8F040005A0E0FF12915543F602AC
:018F0E002240
:10703C0075FFDE75FFAD128EE4E4FFFE0FBF00019D
:10704C000EBE03F8BFE9F51290309005A0EFF012D8
:10705C0090EE128E85D2AF128C941290309005A3C4
:10706C00EFF09005A0E06F60089005A3E09005A0FC
:10707C00F09005A2E060081291E3E49005A2F030D4
:10708C00020A9005A0E0FF128FEEC20230011090B0
:10709C0005A0E0FF7BFF7A91799F128BA9C2017B3F
:1070AC00017A057957128EB8EF60AF900559E0124E
:1070BC004557712E0471760570DD14710F16711A17
:1070CC001770E21A71041B71221D71281E000071C9
:1070DC00C7D2000271C77B017A057957900567EB1F
:1070EC00F0A3EAF0A3E9F01243F5FE9005A0E0FF4F
:1070FC006E60030271C780059005A0E0FF12900F2F
:10710C000271C79005A17401F0C2100271C7E4901E
:10711C0005A1F00271C71291BE0271C71291DD0276
:10712C0071C77B017A05795790056AEBF0A3EAF0F9
:10713C00A3E9F090000312440EFF9005A0E06F70DD
:10714C007AA3E0606E90056AEBF0A3EAF0A3E9F095
:10715C0090000512440EFF90000612440EFD9000A4
:10716C000412440EFB1288CB80497B017A057957B7
:10717C0090056AEBF0A3EAF0A3E9F0900003124447
:10718C000EFF9005A0E06F7032A3E0602690056AB8
:10719C00EBF0A3EAF0A3E9F090000512440EFF9087
:1071AC00000612440EFD90000412440EFB1286C819
:1071BC00128E859005A0E0FF1290519005A1E07011
:1071CC00030270AB900559E014603424FA60531438
:1071DC00700302727C240660030270AB1291447B34
:1071EC00017A057957900567EBF0A3EAF0A3E9F073
:1071FC0090000312440E900512F01291E3806B1272
:10720C0091447B017A057957900567EBF0A3EAF07E
:10721C00A3E9F090000312440E900512F0128E8533
:10722C0080481291447B017A05795790056DEBF0FB
:10723C00A3EAF0A3E9F090000312440EFF900004BF
:10724C0012440EFD90000512440EFBC00390056D18
:10725C00E0FBA3E0FAA3E0F990000612440E9005BF
:10726C008BF0D00312877E128E851291620270AB66
:10727C001291447B017A05795790056DEBF0A3EAE6
:10728C00F0A3E9F090000312440EFF9000041244A6
:10729C000EFD90000512440EFB1279C3128E85125E
:0572AC0091620270ABCD
:035006000289ED2F
:1089ED00C0E0C0F0C083C082C0D075D000C000C050
:1089FD0001C002C003C004C005C006C00775D30086
:108A0D009005A8E014601514601714601914601B0C
:108A1D0014601D2405701C1291E980171274DE80FC
:108A2D0012129196800D1272B180081285F3800397
:108A3D0012911D9005A8E004F0C364809486400255
:108A4D00E4F0D007D006D005D004D003D002D00179
:0D8A5D00D000D0D0D082D083D0F0D0E03255
:10911D009005AAE07003124A031291D79005AAE0B8
:04912D006401F022C7
:108CD900AB84A2AF920AE4FCFDED90062212450E88
:108CE900900624E0FEA3E0780EA60608F6E4F584D3
:108CF900C2AF43B701438F02438F0118E6FE08E66E
:108D0900F5828E83E4F053B7FEF58FA20A92AFAFD6
:038D1900038F8441
:018D1C002234
:024FAA00AB0555
:104FAC00AA84A2AF920BE4FCFDED90062612450EEE
:104FBC00EBFF3395E0FEEFF44E6029900628E0FEFF
:104FCC00A3E07810A60608F6E4F584C2AF43B70157
:104FDC00758F0118E6FC08E6F5828C83EBF053B76D
:0C4FEC00FEE4F58FA20B92AFAF028F84A1
:014FF8002296
:108B480090060AEEF0A3EFF0A3ECF0A3EDF0A3EA91
:108B5800F0A3EBF090060EE07002A3E060429006EE
:108B68000AE0FEA3E0FFA3E0FCA3E0F5828C83E02B
:108B7800FD124FAA90060FE024FFF090060EE03495
:108B8800FFF090060DE004F0700690060CE004F08B
:108B980090060BE004F070BC90060AE004F080B484
:018BA80022AA
:0891A700E4900400F0A3F022A3
:108F3900900400E0FEA3E0FF128CD9900400E0FE4B
:108F4900A3E0FF7C007D007B007A04128B48E4904B
:068F59000400F0A3F02269
:0A896100A905900610EEF0A3EFF058
:10896B00EE54FCFE900400E0FCA3E0FD7002EE6C04
:10897B006057ED4C6003128F39900610E0FEEE54F9
:10898B00FCFE7F00900400F0A3EFF0900612EEF0D7
:10899B00A3EFF0A37400F0A37400F07E0490061212
:1089AB00E475F00112448585F082F583E493FD9024
:1089BB000614E475F00112448585F082F583EDF021
:1089CB00EF1F70011EEF4E70D4900610E0FCA3E079
:1089DB00FDEC5403FC74002DF58274003CF583E927
:0189EB00F09B
:0189EC002268
:108C09009005F5EEF0A3EFF0A3EBF0A3EAF0A3E9EA
:108C1900F09005FA74FFF5F012448545F06026904E
:108C290005F5E475F001124485AFF0FE9005F7E013
:108C3900FBA3E475F001124485A9F0FA1243F5FD8E
:068C490012896180CC22BB
:06503300C2C253E6FD229B
:107B35009005CAE0FFA3E0FCA3E0FDA3E0FBA3E002
:107B4500FAA3E0F9900576E508F0E509A3F09005BC
:067B5500D2E0900578F07B
:107B5B00900570EFF0A3ECF0A3EDF0A3EBF0A3EA2C
:047B6B00F0A3E9F0AA
:107B6F009005797403F0A374E8F0A3E584F0E4F5CD
:107B7F008420C7FDC2C4D2C2D2C5E4FF90064EF026
:107B8F0030C3FDAEC1EE24F8602324F8601F24F843
:107B9F00602F24F8603624F8603A24F87003027CD2
:107BAF004724F87003027C4F2438027C57EF700C87
:107BBF00900570E025E044A0F5C27F03C2C5027CAA
:107BCF005D900571E0F5C27F05027C5D90064E74F5
:107BDF0003F0807AEFB4050B900571A3E0F5C27F37
:107BEF0006806BEF6406703E900578E09005737029
:107BFF000FE0FBA3E475F001124485A9F0FA8008A9
:107C0F00E0FBA3E0FAA3E0F91243F5F5C290057784
:107C1F00E024FFF0900576E034FFF0E07002A3E07F
:107C2F00702C7F078028EFB40706D2C47F09801E0F
:107C3F0090064E7405F0801690064E7404F0800E78
:107C4F0090064E7406F0800690064E7401F0EFB465
:107C5F000904C2C3803690064EE0B4031C90057928
:107C6F0074FFF5F012446F45F0600ED2C4D2C5D246
:107C7F00C2C2C3E490064EF0FF90064EE06008C209
:107C8F00C5D2C4C2C38005C2C3027B8F20C7FD907B
:057C9F00057BE0F58407
:017CA40022BD
:107CA5009005ABEFF0A3ECF0A3EDF0A3EBF0A3EAA6
:047CB500F0A3E9F05F
:107CB9009005B37403F0A374E8F0A3E584F0E4F548
:107CC9008420C7FDD2C2C2C4D2C5E4FF90064EF0DB
:107CD90030C3FDAEC1EE1245577D07007D0A087D10
:107CE9000A107D35187D40207D48287D63307D6BE5
:107CF900387D73407D83507DB55800007D07027D36
:107D0900BBC2C5EF700F9005ABE025E044A0F5C2FA
:107D19007F03027DC1EF64016003027DC19005AB61
:107D2900E025E044A1F5C27F04027DC19005ACE0E5
:107D3900F5C27F05027DC190064E7403F08079EF8C
:107D4900B4050B9005ACA3E0F5C27F06806AEFB4D9
:107D59000606D2C57F018060801890064E7404F033
:107D6900805690064E7406F0804EEFB404047F02EC
:107D7900804690064E7405F0803E9005AEE0FBA368
:107D8900E475F001124485A9F0FAE5C212443B906A
:107D990005B2E024FFF09005B1E034FFF0E0700295
:107DA900A3E07004C2C280107F02800CD2C47F0994
:107DB900800690064E7401F0EFB40904C2C3803600
:107DC90090064EE0B4031C9005B374FFF5F012441D
:107DD9006F45F0600ED2C4D2C5D2C2C2C3E49006C8
:107DE9004EF0FF90064EE06008C2C5D2C4C2C380FF
:0F7DF90005C2C3027CD920C7FD9005B5E0F58413
:017E08002257
:1083F7009005CAEFF09005CDEBF0A3EAF0A3E9F002
:088407009005CBECF0A3EDF0B1
:10840F00750A00543FF50B543F605CC37440950BE5
:10841F00FFE4950AFE9005D0E0FCA3E0FDC39FECBE
:10842F009E50068C088D0980048E088F09127B35AB
:10843F0090064EE060037F02229005CCE02509F004
:10844F009005CBE03508F09005D2E0700B9005CE8B
:10845F00E5088509F012446FC39005D1E09509F046
:10846F009005D0E09508F09005D0E0F508A3E0F571
:10847F0009D3E5099400E50894004070E50994409C
:10848F00E50894005013127B3590064EE060037F91
:10849F000222E4F508F50980D89005CAE0FFA3E0B1
:1084AF00FCA3E0FDA3E0FBA3E0FAA3E0F9900576BF
:1084BF00E4F07440127B5190064EE060037F02227D
:1084CF0074C02509F50974FF3508F5089005CCE04F
:1084DF002440F09005CBE03400F09005D2E070918D
:0E84EF009005CE75F04012446F0284807F002D
:0184FD00225C
:109106009005B1E4F0A304F0127CA590064EE06051
:07911600037F01227F00220C
:1090700090064DEBF07B017A06794D9005D0E4F037
:0A908000A304F0E4A3F01283F7222A
:108FCC00C0079005EBE0FFA3E09005B1CFF0A3EF55
:108FDC00F0D007127CA590064EE060037F01227F43
:028FEC00002261
:10908A00C0079005F3E0FFA3E09005D0CFF0A3EF6F
:0A909A00F0E4A3F0D0071283F722E0
:0E8C4F00900616EBF0A3EAF0A3E9F0A3EDF017
:108C5D00E490061BF0900616E0FBA3E0FAA3E0F902
:108C6D00A3E0900600F090061AE0900601F0E4FFF4
:108C7D00128A6AEFB4FF0D90061BE0FE04F0EEC3FE
:068C8D00940340D17E00BB
:018C930022BE
:0B8EB800900642EBF0A3EAF0A3E9F003
:108EC3007E007F007D101245AE900642E0FBA3E0DA
:108ED300FAA3E0F97D101282ECEF7002FF227F010A
:018EE300226C
:108BA9009005B67422F0A3EFF0A37413F01243F505
:108BB9009005B9F090000112440E9005BAF09000AA
:108BC9000212440E9005BBF090000312440E90056A
:108BD900BCF090000412440E9005BDF090000512FF
:108BE900440E9005BEF090000612440E9005BFF0A9
:108BF9007B017A0579B6E490061AF07D0A028C4F5A
:108FEE0090062A7422F0A3EFF0A37403F0A374FF8B
:108FFE00F07B017A06792AE490061AF07D04028C41
:01900E004F12
:10900F0090062E7422F0A3EFF0A3741CF0A374FF4C
:10901F00F07B017A06792EE490061AF07D04028C1B
:01902F004FF1
:10905100E4900632F0A3EFF0A3740AF0A3EFF07BE3
:0F906100017A067932E490061AF07D04028C4FF2
:1080E400420405000042040A000042040C0000C1DE
:0580F40004C105C103F9
:0A918C00C205C204E490044EF02274
:108F5F00E4900405F0A3F090040AF0A3F090040E3F
:108F6F00F090040CF0A3F0900408F0A37440F0E428
:058F7F00900407F02240
:0691C50012918C028F5F85
:1090BD00E4F5848FC343C30175C04475CF8EC2C31D
:0990CD0043E60290040304F022C2
:10914400E4F58420C7FDC2C21291C5E4900403F083
:0191540022F8
:0B916200E4F584D2C290040304F02264
:0D915500AE071290BD900404EFF00291C52A
:108F8400E4900645F0A3F0300502FF222004FDD250
:108F94000590044FE4F0A37410F0900452EFF0E451
:048FA400A3F07F01B6
:018FA80022A6
:108E510030050A90044FE07002A3E070037F002206
:108E6100900450E024FFF090044FE034FFF09004B0
:108E710053E0FE04F074542EF582E43404F583EFDC
:048E8100F07F01225B
:0B916D00300507C205D2041250092291
:0E500900AF84E4F58420C7FDC2C4D2C58F84F5
:015017002276
:108A6A009005FDEBF0A3EAF0A3E9F0900403E070AF
:108A7A0002FF22900600E0FE6005D3941040037FB7
:088A8A000022128F84EF604E00
:108A9200E4900602F0900600E0FF900602E0FEC3BA
:108AA2009F50249005FDE0FBA3E0FAA3E0F98E823B
:108AB20075830012440EFF128E51EF7002FF229056
:108AC2000602E004F080CEE490044EF012916D9024
:0E8AD2000601E070032004FD90044EE0FF2238
:038AE0007FFF22F3
:0E82EC00900636EBF0A3EAF0A3E9F0A3EDF064
:1082FA00E4FFD3900406E09400900405E0648094BF
:10830A008050012253E6FD90040CE0FEA3E0240E07
:10831A00F58274043EF583E0FF90040CE475F001E5
:10832A0012446FFCE5F064404C700690040CF0A314
:10833A00F0900409E004F07006900408E004F0E408
:10834A00FE900639E0FDEEC39D5054EEC39F504F98
:10835A0090040CE0FCA3E0240EF58274043CF5833F
:10836A00E0FD900636E0FBA3E0FAA3E0F98E827501
:10837A008300ED12444D90040CE475F00112446F31
:10838A00FCE5F064404C700690040CF0A3F09004F5
:10839A0009E004F07006900408E004F00E80A2EEF2
:1083AA00C39F502990040CE475F00112446FFCE558
:1083BA00F064404C700690040CF0A3F0900409E0BD
:1083CA0004F07006900408E004F00E80D2900406CF
:1083DA00E024FFF0900405E034FFF043E602900643
:0C83EA0039E0FEEFC39E50028002AF0697
:0183F6002264
:1090D600D3900406E09400900405E06480948040F8
:0890E600047F0180027F0022DB
:03501800027E090C
:107E0900C0E0C0F0C083C082C0D075D000C000C03F
:037E190006C00799
:107E1C00C20CAFC1EF1245577E52087E52107E62E3
:107E2C00187E67207E74287EA1307EAC387EB460CC
:107E3C007EAF687EB4707EAF787EBC807EBC907F57
:107E4C0033A000007F41900452E0F5C2C2C59004FB
:107E5C0051E4F0027F43900453802890044E74FD4B
:107E6C00F0D2C4D2C5027F43900453E0FF9004517A
:107E7C00E0C39F5014E0FF04F074542FF582E434F7
:107E8C0004F583E0F5C2027F43D2C490044EE4F0C3
:107E9C00C204027F43D2C590044E74FEF0027F43AD
:107EAC00027F38D203027F43900402E4F0027F4346
:107EBC00900402E07020E5C2F0E0FFC3900409E0FA
:107ECC009F7480F8900408E06480985003128F5FD0
:107EDC00900402E004F0900409E024FFF090040800
:107EEC00E034FFF090040AE0FEA3E0240EF5827467
:107EFC00043EF583E5C2F090040AE475F0011244E7
:107F0C006FFEE5F064404E700690040AF0A3F0900A
:107F1C000402E014F07020900406E004F070189055
:107F2C000405E004F0801030030DC203900451E40A
:107F3C00F0D2C58002D20C300C0EC2C6D2C6C2C55D
:0A7F4C00C2C4D2C2C20CC204C2C3F8
:107F5600D007D006D000D0D0D082D083D0F0D0E0E9
:017F660032E8
:0591CB00A2C7E433FF20
:0191D000227C
:1080F9004104A0004104A1004104A2004104A300DD
:108109004A04A400000002000400060007410464B8
:018119000164
:0491E90043E8102225
:09919600758402D2ECE4F5842298
:035030000284FEF9
:1084FE00C0E0C083C082C0D075D000C004C005C02B
:10850E0006C00753E8DFAFBFEFFEADBE7C00E42D23
:10851E00FFEC3E90049DF0A3EFF090049DE0FCA3D1
:10852E00E0FD9004A0E0FF3395E0FEEF25E0FFEEC6
:10853E0033FE74A42FF58274043EF583A3E025E088
:10854E00FF0582D5820215831582E033FE74712FEA
:10855E00F58274043EF583ECF0A3EDF09004A0E0F8
:10856E0004F0C364809485404DE4F0900471E0FF04
:10857E00A3E0900491CFF0A3EFF0900475E0FFA379
:10858E00E0900493CFF0A3EFF0900479E0FFA3E026
:10859E00900495CFF0A3EFF090047DE0FFA3E09060
:1085AE000499CFF0A3EFF090047FE0FFA3E09004D6
:1085BE009BCFF0A3EFF09004A0E0FF3395E0FEEF29
:1085CE0025E0FFEE33FE74A42FF58274043EF5838E
:1085DE00A3E0F5BBD007D006D005D004D0D0D08212
:0585EE00D083D0E03253
:03503900027825D5
:10782500C0E0C0F0C083C082C0D075D000C000C029
:0D78350001C002C003C004C005C006C007AA
:1078420075840253E8DFC2ED90049FE5BEF0E07557
:10785200F010A4FD9004A1E0FF3395E0FEEF25E0D7
:10786200FFEE33FE74812FF58274043EF583E5F05A
:10787200F0A3EDF09004A1E004F0C364809488507A
:107882000302799F7401F090048FE0FFA3E090045B
:1078920097CFF0A3EFF0900483E0FFA3E09004659C
:1078A200CFF0A3EFF0900485E0FFA3E0900467CF50
:1078B200F0A3EFF0900487E0FFA3E0900469CFF01B
:1078C200A3EFF0900489E0FFA3E090046BCFF0A354
:1078D200EFF090048BE0FFA3E090046DCFF0A3EFF4
:1078E200F090048DE0FFA3E090046FCFF0A3EFF0DF
:1078F200900464E06041E4FDFCED25E0FFEC33FE22
:1079020074652FF58274043EF583E0FAA3E0FB74FC
:107912007C2FF58274053EF583EAF0A3EBF00DBDF2
:1079220000010CED64064C70D0900464E004F0E0B9
:10793200D3940A4002E4F0900464E070047D018074
:10794200027D007F001246A8900464E070047D016D
:1079520080027D007F011246A8900464E070047DDD
:107962000180027D007F021246A8900464E0700448
:107972007D0180027D007F031246A8900464E070BE
:10798200047D0180027D007F041246A8900464E019
:1079920070047D0180027D007F051246A89004A13B
:0679A200E0F5BB75840056
:1079A800D007D006D005D004D003D002D001D00033
:0B79B800D0D0D082D083D0F0D0E032DD
:10811A00C108C1094105408041054180420542002C
:10812A000043054A00000043054D00000043055086
:10813A000000004305530000004105560041053D7B
:01814A000133
:10903000E5B0A2E29206E5B0A2E39207300609305D
:1090400007037F66227F67223007037F68227F69DC
:0190500022FD
:104A0300900540E0A3F0E5B05402900540F0A3E028
:104A1300FD900540E0FE6D900536F0EE701DED60F3
:104A230005E4900556F0900556E004F0E0D394D0E9
:104A33004037200902D201D209802E900541E0704F
:104A430028900556E0C394D0501D3000099005A16D
:104A5300E06401F080119005A1E0600B9005A27461
:104A630001F0E49005A1F0C209E490064FF090062E
:104A73004FE0FFD3648094824003024BA0E0FEFD2D
:104A83003395E0FC744A2DF58274053CF583E0FB15
:104A9300744D2DF58274053CF583EBF0EE2404FE92
:104AA3007401A806088002C333D8FC55A0FEEFFDAD
:104AB3003395E0FC744A2DF58274053CF583EEF0E2
:104AC30090053DE06018744A2DF58274053CF5832A
:104AD300E0FF744D2DF58274053CF583EFF09006ED
:104AE3004FE0FFFD3395E0FC744D2DF58274053CDA
:104AF300F583E0FE744A2DF58274053CF583E06E80
:104B0300FEEF3395E0FC74372DF58274053CF58395
:104B1300EEF0744A2DF58274053CF583E07042741F
:104B23004D2DF58274053CF583E06007E490054262
:104B3300F0A3F0900543E004F07006900542E00412
:104B4300F0D3900543E094F0900542E09400404494
:104B530090053FE070031291AF90053F7401F08020
:104B63003390064FE0FFFD3395E0FC744D2DF58245
:104B730074053CF583E0701CC3900543E094C0903A
:104B83000542E094005008EF3395E0FE128F0FE4E6
:104B930090053FF090064FE004F0024A7190064FF3
:104BA3007402F090064FE0FFC364809480500302C8
:104BB3004CEBE0FEFD3395E0FC74502DF58274055B
:104BC3003CF583E0FB74532DF58274053CF583EBD0
:104BD300F0EE2404FE7401A806088002C333D8FC57
:104BE30055B0FEEFFD3395E0FC74502DF58274054E
:104BF3003CF583EEF090053DE0601874502DF5828E
:104C030074053CF583E0FF74532DF58274053CF580
:104C130083EFF090064FE0FFFD3395E0FC74532DD6
:104C2300F58274053CF583E0FE74502DF58274051E
:104C33003CF583E06EFEEF3395E0FC743A2DF5828C
:104C430074053CF583EEF074502DF58274053CF544
:104C530083E0704E74532DF58274053CF583E06058
:104C63001E90064FE0FF3395E0FEEF25E0FFEE33A5
:104C7300FE74442FF58274053EF583E4F0A3F090AF
:104C8300064FE0FF3395E0FEEF25E0FFEE33FE74C1
:104C9300442FF58274053EF583E475F00112446FE9
:104CA300803D74532DF58274053CF583E07030909C
:104CB300064FE0FD3395E0FCED25E0FFEC33FE7499
:104CC300442FF58274053EF583E0FEA3E0C394C050
:104CD300EE9400500AAF05AE04128E18128FA990FD
:104CE300064FE014F0024BA690053DE06002E4F0AD
:014CF300229E
:0691D10030313234353666
:1085F300E4FDFCC3ED9403EC648094805023ED25EB
:10860300E0FFEC33FE74942FF58274053EF583A3EB
:10861300E0C4F8540FC868FF0582D5820215838031
:108623002CC3ED9406EC64809480502FED25E0FF7D
:10863300EC33FE74A92FF58274043EF583A3E0C4E2
:10864300F8540FC868FF0582D5820215831582E0AE
:10865300C454F048900647F0A3EFF074D12DF5828F
:1086630074913CF583E493FFE4F584C2FA8F9B3065
:10867300FFFDC2FFE4FFFE0FBF00010EEF64324EA9
:1086830070F5900647E0F59B30FFFDC2FFE4FEFF67
:108693000FBF00010EEF64324E70F5900648E0F50F
:1086A3009B30FFFDC2FFE4FEFF0FBF00010EEF642E
:1086B300324E70F5D2FA0DBD00010CED64064C602C
:0486C300030285F633
:0186C7002290
:1046A80090FFFF12457DEDF090FFFF12457DEFF082
:0646B80090FFEE12457DAB
:1046BE00850C83850D82E4F0A3F09000121245A1C3
:1046CE00E025E0247CF582E43405F583E0FEA3E0EA
:1046DE00FFFBAA06E4F9F89000121245A1E025E0CE
:1046EE002465F582E43404F583E0FEA3E0FFC3EF16
:1046FE009BFFEE9AFEE499FDE498FC850C83850DF4
:10470E0082A3A312450EE47F40FEFDFC850C83853B
:10471E000D82A3A3E0F8A3E0F9A3E0FAA3E0FBC3A4
:10472E001244F8400B850C83850D82E4F0A304F04F
:10473E0074FF7FC0FEFDFC850C83850D82A3A3E074
:10474E00F8A3E0F9A3E0FAA3E0FBD31244F8500B70
:10475E00850C83850D8274FFF0A3F0850C83850D87
:10476E0082E0FEA3E0FF4E70030249FDEFF47002FB
:07477E00EEF4600302488A1B
:104785009000121245A1E025E0247CF582E4340571
:10479500F583E0FEA3E0FFE4FCFD90000E1245A1C9
:1047A50012450EE47F01FEFDFC90000E1245A1E0CE
:1047B500F8A3E0F9A3E0FAA3E0FBC31244F8500D17
:1047C50090000E1245A112451A000000019000123A
:1047D5001245A1E025E02417F582E43405F583E0D0
:1047E500FEA3E0FFE4FCFD7BFF7A0FF9F812449B82
:1047F50090000E1245A1E0F8A3E0F9A3E0FAA3E0CA
:10480500FB128D1D9000061245A112450E90001257
:104815001245A1E025E02465F582E43404F583E042
:10482500FEA3E0FFE4FCFD9000061245A1E0F8A31D
:10483500E0F9A3E0FAA3E0FB12449B90000A1245BD
:10484500A112450EE47BFF7A0FF9F890000A124594
:10485500A1E0FCA3E0FDA3E0FEA3E0FF128D1D9007
:1048650000121245A1E025E02417F582E43405F590
:1048750083EEF0A3EFF09000131245A1E070030260
:0248850049D414
:104887000249D1850C83850D82E0FEA3E064014EC9
:0548970060030249D49A
:10489C009000121245A1E025E02417F582E43405BE
:1048AC00F583E0FEA3E0FBC374FF9BFF740F9EFE39
:1048BC00E49400FDE49400FCE47BFF7A0FF9F81219
:1048CC00449B9000061245A112450E900012124511
:1048DC00A1E025E0247CF582E43405F583E0FEA319
:1048EC00E0FBC374FF9BFF740F9EFEE49400FDE499
:1048FC009400FC90000A1245A112450EE47F01FEC3
:10490C00FDFC90000A1245A1E0F8A3E0F9A3E0FA3F
:10491C00A3E0FBC31244F8500D90000A1245A112FB
:10492C00451A000000019000061245A1C083C08208
:10493C00E0FCA3E0FDA3E0FEA3E0FF90000A12451B
:10494C00A1E0F8A3E0F9A3E0FAA3E0FB128D1DD0DF
:10495C0082D08312450E9000121245A1E025E0246E
:10496C0065F582E43404F583E0FEA3E0FBC374FF39
:10497C009BFF740F9EFEE49400FDE49400FC9000F9
:10498C00061245A1E0F8A3E0F9A3E0FAA3E0FB12BC
:10499C00449BE47BFF7A0FF9F8128D1DC374FF9FC3
:1049AC00FF740F9EFE9000121245A1E025E0241723
:1049BC00F582E43405F583EEF0A3EFF090001312CA
:0849CC0045A1E06003128FA970
:1049D4009000121245A1E0FF25E02465F582E4343D
:1049E40004F583E0FCA3E0FDEF25E0247CF582E4FC
:0949F4003405F583ECF0A3EDF0AD
:0649FD0090001402457D4C
:10814B004304EB0002044304EE04000C4304F10669
:10815B00020E4304F405010D4304F707030F430418
:10816B00FA090A0B4304FD0B0F074305000A0E0621
:10817B00430503090D05430506080C0443050903D4
:10818B00020142050C000042050E0000C10D430424
:0F819B00E51919194304E81010104205100000EF
:104CF40090050CE0FFA3E090063ACFF0A3EFF0E4B8
:104D040090050CF0A3F0FDED25E024AFF582E4342A
:104D140004F583E0FEC3EE940F401F74EE2DF5827C
:104D2400E43404F583E0FF74017E00A807088005DD
:104D3400C333CE33CED8F9024DDEED25E024AFF5F2
:104D440082E43404F583E0FEA3E0C394FFEE940907
:104D5400401E74F42DF582E43404F583E0FF7401FD
:104D64007E00A807088005C333CE33CED8F9806A05
:104D7400ED25E024AFF582E43404F583E0FEA3E0FE
:104D8400C394FFEE9406401E74F12DF582E43404BE
:104D9400F583E0FF74017E00A807088005C333CEC5
:104DA40033CED8F98034ED25E024AFF582E4340421
:104DB400F583E0FEA3E0C394FFEE9403402774F769
:104DC4002DF582E43404F583E0FF74017E00A80726
:104DD400088005C333CE33CED8F9FF90050CE04EDE
:104DE400F0A3E04FF0ED25E0249AF582E43405F5D4
:104DF40083E0FEA3E064024E7042EDFFC374029FA1
:104E0400FFE49400FE74FA2FF58274043EF583E007
:104E1400FF74017E00A807088005C333CE33CED8C3
:104E2400F9FF90050CE04EF0A3E04FF074E52DF58A
:104E340082E43404F5837419F0024EF6ED25E0247F
:104E44009AF582E43405F583E0FEA3E064014E6044
:104E540003024EF674E52DF582E43404F583E06034
:104E64004374E52DF582E43404F583E014F06034F2
:104E7400EDFFC374029FFFE49400FE74FA2FF582E1
:104E840074043EF583E0FF74017E00A807088005E2
:104E9400C333CE33CED8F9FF90050CE04EF0A3E037
:104EA4004FF0804E74E82DF582E43404F583E01469
:104EB400F0703FEDFFC374029FFFE49400FE74FAA8
:104EC4002FF58274043EF583E0FF74017E00A80789
:104ED400088005C333CE33CED8F9FF90050CE04EDD
:104EE400F0A3E04FF074E82DF582E43404F5837404
:0D4EF40010F00DED64036003024D0BC2B021
:104F010090063CE4F0A37410F090063C74FFF5F0B9
:0E4F1100124485FED3E5F09400EE940050EBC0
:104F1F00E4FD90050CE0FEA3E0A805088005CEC3D4
:0A4F2F0013CE13D8F9139286C2873F
:104F390090063CE4F0A37410F090063C74FFF5F081
:0E4F4900124485FED3E5F09400EE940050EB88
:024F5700D287FF
:104F590090063CE4F0A37410F090063C74FFF5F061
:0E4F6900124485FED3E5F09400EE940050EB68
:0B4F7700ED64076004EDB40F20D2B021
:104F820090063CE4F0A37410F090063C74FFF5F038
:0E4F9200124485FED3E5F09400EE940050EB3F
:094FA0000DED64106003024F21C5
:014FA90022E5
:10768300E490050EF0A3F0FD74132DF582E43405A8
:10769300F583E01460251460402402706374FD2DAB
:1076A300F582E43404F583E0FF74017E00A8070843
:1076B3008005C333CE33CED8F9803A74002DF582DA
:1076C300E43405F583E0FF74017E00A80708800514
:1076D300C333CE33CED8F9801C74032DF582E43442
:1076E30005F583E0FF74017E00A807088005C33316
:1076F300CE33CED8F9FF90050EE04EF0A3E04FF065
:10770300900516E0602774062DF582E43405F583B1
:10771300E0FF74017E00A807088005C333CE33CE93
:10772300D8F9FF90050EE04EF0A3E04FF074232D3F
:10773300F582E43405F583E0602774092DF582E4CE
:107743003405F583E0FF74017E00A807088005C3B4
:1077530033CE33CED8F9FF90050EE04EF0A3E04FC1
:10776300F09005A1E0600790050FE04401F00DEDF6
:097773006403600302768BC2A2DC
:10777C00900649E4F0A37410F090064974FFF5F0FC
:0E778C00124485FED3E5F09400EE940050EB1D
:10779A00E4FD90050EE0FEA3E0A805088005CEC32F
:0A77AA0013CE13D8F91392A0C2A168
:1077B400900649E4F0A37410F090064974FFF5F0C4
:0E77C400124485FED3E5F09400EE940050EBE5
:0277D200D2A142
:1077D400900649E4F0A37410F090064974FFF5F0A4
:0E77E400124485FED3E5F09400EE940050EBC5
:0B77F200ED64076004EDB40F20D2A28C
:1077FD00900649E4F0A37410F090064974FFF5F07B
:0E780D00124485FED3E5F09400EE940050EB9B
:09781B000DED6410600302779C7E
:017824002241
:0691D700124CF402768345
:108F0F0074132FF58274053EF583E004F074132F6C
:108F1F00F58274053EF583E0D39402400C74132F51
:0A8F2F00F58274053EF583E4F0229C
:108E1800C374029FFDE49EFC74232DF58274053C07
:108E2800F583E004F074232DF58274053CF583E0A6
:108E3800D39401401374029FFFE49EFE74232FF520
:098E48008274053EF583E4F0227A
:0891AF00900516E06401F022B6
:1081AA004105120043051300000041051600C110E5
:0481BA004105260055
:0691DD00E4900526F022DB
:0791BE009005267401F02268
:108832001291A7E4900650F0900650E0FFC3940610
:108842005018EF25E02417F582E43405F583E4F0AF
:10885200A3F0900650E004F080DEE4900650F09021
:108862000650E0FFD39402502074232FF582E434A3
:1088720005F583E4F074132FF582E43405F583E4FF
:10888200F0900650E004F080D6E4900516F09006D1
:1088920050F0900650E0FFC3941E502A75F00FEF7F
:1088A200A42402F582E5F034F0AF82FE7B017A0562
:1088B20079179005FAE4F0A3740FF0128C09900670
:0988C20050E004F080CC028F3973
:108DA20090064B7402F0E4A3F01291A77EF07F01CB
:108DB2007B017A06794B9005FAE4F0A304F0128C59
:108DC200097EF07F007B017A06794C9005FAE4F087
:0C8DD200A304F0128C09128F39028832C1
:108FA9003000142010119005A1E0600B900526E017
:108FB9007002D202D210222000089005A1E07002AE
:038FC90004F0228F
:1090EE0090F000E493F46007A3E49364026003122B
:0890FE008DA2E4900512F0229E
:108E8500A2AF920EC2AF900512E0FFC3941E501E12
:108E9500EF75F00FA42402F974F035F0FA7BFF7832
:108EA500177C057D017E007F0F1243CFC210A20EF5
:028EB50092AF7A
:018EB7002298
:108D6100A2AF920FC2AF900512E0C3941E502B1216
:108D710091A7900512E075F00FA42402F582E5F0A9
:108D810034F0AF82FE7B017A0579179005FAE4F0A1
:108D9100A3740FF0128C09128F39C210A20F92AF77
:018DA10022AF
:0691E300128D61C2102292
:05877E00900589EDF0FB
:1087830090058BE004F090058EEFF0A3EBF09005DD
:1087930089E0FF90058EE0FED39F40030288317588
:1087A300F00FEEA42402F582E5F034F0AF829005D9
:1087B30090F0A3EFF090058FE075F00FA42402F57D
:1087C30082E5F034F0AF82900592F0A3EFF0E490ED
:1087D300058CF0A3F0900592E475F001124485AF87
:1087E300F0FE900590E0FCA3E0F5828C83E493FD1A
:1087F300128961900591E004F07006900590E00401
:10880300F090058DE004F0700690058CE004F0C351
:1088130090058DE0940F90058CE0940040B7128F83
:0E8823003990058EE004F0A3E004F002879186
:018831002224
:0579C3009005D3EDF07A
:1079C8009005D8EFF0A3EBF09005D3E0FF9005D831
:1079D800E0D39F4003027B34A3E075F00FA4240298
:1079E800F582E5F034F0AF829005D4F0A3EFF0E42F
:1079F8009005DAF0A3F09005DAE0FEA3E0FFC39467
:107A08000FEE940050389005D4E0FCA3E0F5828C8A
:107A180083E493FD74272FF582E43405F583EDF0B4
:107A28009005D5E004F070069005D4E004F09005C8
:107A3800DBE004F070C09005DAE004F080B890054F
:107A4800D8E075F00FA42402F582E5F034F0AF8297
:107A58009005D6F0A3EFF09005D9E075F00FA424B7
:107A680002F582E5F034F0AF829005D4F0A3EFF090
:107A7800E49005DAF0A3F09005D4E475F00112441F
:107A880085AFF0FE9005D6E0FCA3E0F5828C83E498
:107A980093FD1289619005D7E004F070069005D631
:107AA800E004F09005DBE004F070069005DAE004ED
:107AB800F0C39005DBE0940F9005DAE0940040B73E
:107AC8009005D8E075F00FA42402F582E5F034F0B3
:107AD800AF829005D6F0A3EFF0E49005DAF0A3F0BA
:107AE8009005DAE0FCA3E0FDC3940FEC9400502C61
:107AF8009005D6E475F001124485AFF0FE74272D89
:107B0800F582E43405F583E0FD1289619005DBE038
:107B180004F070CC9005DAE004F080C4128F39903C
:0C7B280005D8E004F0A3E004F00279D0DE
:017B3400222E
:0B86C8009005C0EFF0A3EDF0A3EBF075
:1086D300A2AFE433A3F0C2AF1250339005C1E0FE62
:1086E3009005C0E0FDEDFF9005C8EEF0A3EFF0E4C8
:1086F3009005C4F09005C2E0FF9005C8E0FCA3E03C
:10870300FD7B017A0579279005EBE4F0A3740FF064
:10871300128FCC9005C9E0240FF09005C8E0340017
:10872300F09005C4E075F00FA42402F974F035F05D
:10873300FAA374FFF0A3EAF0A3E9F01291A790055E
:10874300C5A3E0FAA3E0AE02FF7B017A0579279087
:1087530005FAE4F0A3740FF0128C09128F39900517
:10876300C4E004F0E0C3941E408A9005A0E0FF1229
:0A87730091559005C3E024FF92AF7A
:01877D0022D9
:0B88CB009005DCEFF0A3EDF0A3EBF054
:1088D600A2AFE433A3F0C2AF1250339005DDE0FE41
:1088E6009005DCE0FDEDFF9005E1EEF0A3EFF0E48E
:1088F6009005E0F09005E0E0FFC3941E504C75F043
:108906000FEFA42402F582E5F034F0AF82FE900565
:10891600E3F0FAA3EFF0FB9005DEE0FF9005E1E05F
:10892600FCA3E0FDA9037BFF9005F3E4F0A3740F1D
:10893600F012908A9005E2E0240FF09005E1E03411
:1089460000F09005E0E004F080AA9005A0E0FF1298
:0A89560091559005DFE024FF92AF79
:0189600022F4
:10503C0000C800C700C700C700C700C700C700C62C
:10504C0000C600C600C600C600C600C600C500C526
:10505C0000C500C500C500C500C500C400C400C41F
:10506C0000C400C400C400C400C300C300C300C318
:10507C0000C300C300C300C200C200C200C200C211
:10508C0000C200C100C100C100C100C100C100C10B
:10509C0000C000C000C000C000C000C000C000BF05
:1050AC0000BF00BF00BF00BF00BF00BF00BE00BEFE
:1050BC0000BE00BE00BE00BE00BE00BD00BD00BDF7
:1050CC0000BD00BD00BD00BD00BC00BC00BC00BCF0
:1050DC0000BC00BC00BB00BB00BB00BB00BB00BBEA
:1050EC0000BB00BA00BA00BA00BA00BA00BA00BAE3
:1050FC0000B900B900B900B900B900B900B900B8DD
:10510C0000B800B800B800B800B800B800B700B7D5
:10511C0000B700B700B700B700B600B600B600B6CF
:10512C0000B600B600B600B500B500B500B500B5C8
:10513C0000B500B500B400B400B400B400B400B4C1
:10514C0000B400B300B300B300B300B300B300B3BA
:10515C0000B200B200B200B200B200B200B200B1B4
:10516C0000B100B100B100B100B100B000B000B0AE
:10517C0000B000B000B000B000AF00AF00AF00AFA7
:10518C0000AF00AF00AF00AE00AE00AE00AE00AEA0
:10519C0000AE00AE00AD00AD00AD00AD00AD00AD99
:1051AC0000AD00AC00AC00AC00AC00AC00AC00AB93
:1051BC0000AB00AB00AB00AB00AB00AB00AA00AA8D
:1051CC0000AA00AA00AA00AA00AA00A900A900A986
:1051DC0000A900A900A900A900A800A800A800A87F
:1051EC0000A800A800A800A700A700A700A700A778
:1051FC0000A700A700A600A600A600A600A600A671
:10520C0000A500A500A500A500A500A500A500A46B
:10521C0000A400A400A400A400A400A400A300A364
:10522C0000A300A300A300A300A300A200A200A25D
:10523C0000A200A200A200A200A100A100A100A156
:10524C0000A100A100A000A000A000A000A000A050
:10525C0000A0009F009F009F009F009F009F009F49
:10526C00009E009E009E009E009E009E009E009D43
:10527C00009D009D009D009D009D009D009C009C3C
:10528C00009C009C009C009C009C009B009B009B35
:10529C00009B009B009B009A009A009A009A009A2F
:1052AC00009A009A00990099009900990099009928
:1052BC000099009800980098009800980098009821
:1052CC00009700970097009700970097009700961B
:1052DC000096009600960096009600960095009514
:1052EC00009500950095009500940094009400940E
:1052FC000094009400940093009300930093009307
:10530C0000930093009200920092009200920092FF
:10531C0000920091009100910091009100910091F8
:10532C00009000900090009000900090008F008FF3
:10533C00008F008F008F008F008F008E008E008EEC
:10534C00008E008E008E008E008D008D008D008DE5
:10535C00008D008D008D008C008C008C008C008CDE
:10536C00008C008C008B008B008B008B008B008BD7
:10537C00008B008A008A008A008A008A008A0089D1
:10538C0000890089008900890089008900880088CB
:10539C0000880088008800880088008700870087C4
:1053AC0000870087008700870086008600860086BD
:1053BC0000860086008600850085008500850085B6
:1053CC0000850084008400840084008400840084B0
:1053DC0000830083008300830083008300830082AA
:1053EC0000820082008200820082008200810081A3
:1053FC00008100810081008100810080008000809C
:10540C000080008000800080007F007F007F007F94
:10541C00007F007F007E007E007E007E007E007E8E
:10542C00007E007D007D007D007D007D007D007D87
:10543C00007C007C007C007C007C007C007C007B81
:10544C00007B007B007B007B007B007B007A007A7A
:10545C00007A007A007A007A007900790079007974
:10546C00007900790079007800780078007800786D
:10547C000078007800770077007700770077007766
:10548C00007700760076007600760076007600765F
:10549C000075007500750075007500750075007459
:1054AC000074007400740074007400730073007353
:1054BC00007300730073007300720072007200724C
:1054CC000072007200720071007100710071007145
:1054DC00007100710070007000700070007000703E
:1054EC000070006F006F006F006F006F006F006E38
:1054FC00006E006E006E006E006E006E006D006D32
:10550C00006D006D006D006D006D006C006C006C2A
:10551C00006C006C006C006C006B006B006B006B23
:10552C00006B006B006B006A006A006A006A006A1C
:10553C00006A006A00690069006900690069006915
:10554C000068006800680068006800680068006710
:10555C000067006700670067006700670066006609
:10556C000066006600660066006600650065006502
:10557C0000650065006500650064006400640064FB
:10558C0000640064006400630063006300630063F4
:10559C0000630063006300630063006300620062E9
:1055AC0000620062006200620062006200620062DF
:1055BC0000620061006100610061006100610061D6
:1055CC0000610061006100610061006000600060CA
:1055DC0000600060006000600060006000600060BF
:1055EC00005F005F005F005F005F005F005F005FB7
:1055FC00005F005F005F005E005E005E005E005EAC
:10560C00005E005E005E005E005E005E005E005D9F
:10561C00005D005D005D005D005D005D005D005D96
:10562C00005D005D005C005C005C005C005C005C8C
:10563C00005C005C005C005C005C005B005B005B81
:10564C00005B005B005B005B005B005B005B005B76
:10565C00005B005A005A005A005A005A005A005A6D
:10566C00005A005A005A005A005900590059005962
:10567C000059005900590059005900590059005956
:10568C00005800580058005800580058005800584E
:10569C000058005800580057005700570057005743
:1056AC000057005700570057005700570056005638
:1056BC00005600560056005600560056005600562E
:1056CC000056005600550055005500550055005524
:1056DC000055005500550055005500540054005419
:1056EC00005400540054005400540054005400540E
:1056FC000053005300530053005300530053005306
:10570C0000530053005300530052005200520052F9
:10571C0000520052005200520052005200520051EE
:10572C0000510051005100510051005100510051E5
:10573C0000510051005000500050005000500050DB
:10574C00005000500050005000500050004F004FCF
:10575C00004F004F004F004F004F004F004F004FC5
:10576C00004F004E004E004E004E004E004E004EBC
:10577C00004E004E004E004E004E004D004D004DB0
:10578C00004D004D004D004D004D004D004D004DA5
:10579C00004C004C004C004C004C004C004C004C9D
:1057AC00004C004C004C004B004B004B004B004B92
:1057BC00004B004B004B004B004B004B004B004A86
:1057CC00004A004A004A004A004A004A004A004A7D
:1057DC00004A004A00490049004900490049004973
:1057EC000049004900490049004900480048004868
:1057FC00004800480048004800480048004800485D
:10580C000048004700470047004700470047004753
:10581C000047004700470047004600460046004648
:10582C00004600460046004600460046004600463C
:10583C000045004500450045004500450045004534
:10584C000045004500450044004400440044004429
:10585C00004400440044004400440044004300431E
:10586C000043004300430043004300430043004314
:10587C00004300430042004200420042004200420A
:10588C0000420042004200420042004100410041FF
:10589C0000410041004100410041004100410041F4
:1058AC0000400040004000400040004000400040EC
:1058BC000040004000400040003F003F003F003FE0
:1058CC00003F003F003F003F003F003F003F003ED5
:1058DC00003E003E003E003E003E003E003E003ECC
:1058EC00003E003E003D003D003D003D003D003DC2
:1058FC00003D003D003D003D003D003D003C003CB6
:10590C00003C003C003C003C003C003C003C003CAB
:10591C00003C003B003B003B003B003B003B003BA2
:10592C00003B003B003B003B003B003A003A003A96
:10593C00003A003A003A003A003A003A003A003A8B
:10594C000039003900390039003900390039003983
:10595C000039003900390038003800380038003878
:10596C00003800380038003800380038003800376C
:10597C000037003700370037003700370037003763
:10598C000037003700360036003600360036003659
:10599C00003600360036003600360035003500354E
:1059AC000035003500350035003500350035003543
:1059BC00003500340034003400340034003400343A
:1059CC00003400340034003400330033003300332F
:1059DC000033003300330033003300330033003224
:1059EC00003200320032003200320032003200321B
:1059FC000032003200320031003100310031003110
:105A0C000031003100310031003100310030003004
:105A1C0000300030003000300030003000300030FA
:105A2C0000300030002F002F002F002F002F002FF0
:105A3C00002F002F002F002F002F002E002E002EE5
:105A4C00002E002E002E002E002E002E002E002EDA
:105A5C00002D002D002D002D002D002D002D002DD2
:105A6C00002D002D002D002D002C002C002C002CC6
:105A7C00002C002C002C002C002C002C002C002BBB
:105A8C00002B002B002B002B002B002B002B002BB2
:105A9C00002B002B002A002A002A002A002A002AA8
:105AAC00002A002A002A002A002A002A002900299C
:105ABC000029002900290029002900290029002992
:105ACC000029002800280028002800280028002889
:105ADC00002800280028002800280027002700277D
:105AEC000027002700270027002700270027002772
:105AFC000027002700270027002700270027002762
:105B0C000027002700270027002700270027002751
:105B1C000027002700270027002700270027002642
:105B2C000026002600260026002600260026002639
:105B3C000026002600260026002600260026002629
:105B4C000026002600260026002600260026002619
:105B5C000026002600260026002600260026002609
:105B6C000026002500250025002500250025002500
:105B7C0000250025002500250025002500250025F1
:105B8C0000250025002500250025002500250025E1
:105B9C0000250025002500250025002500250025D1
:105BAC0000250025002500240024002400240024C6
:105BBC0000240024002400240024002400240024B9
:105BCC0000240024002400240024002400240024A9
:105BDC000024002400240024002400240024002499
:105BEC00002400240024002400240023002300238C
:105BFC000023002300230023002300230023002381
:105C0C000023002300230023002300230023002370
:105C1C000023002300230023002300230023002360
:105C2C000023002300230023002300230023002251
:105C3C000022002200220022002200220022002248
:105C4C000022002200220022002200220022002238
:105C5C000022002200220022002200220022002228
:105C6C000022002200220022002200220022002218
:105C7C00002200210021002100210021002100210F
:105C8C000021002100210021002100210021002100
:105C9C0000210021002100210021002100210021F0
:105CAC0000210021002100210021002100210021E0
:105CBC0000210021002100200020002000200020D5
:105CCC0000200020002000200020002000200020C8
:105CDC0000200020002000200020002000200020B8
:105CEC0000200020002000200020002000200020A8
:105CFC0000200020002000200020001F001F001F9B
:105D0C00001F001F001F001F001F001F001F001F8F
:105D1C00001F001F001F001F001F001F001F001F7F
:105D2C00001F001F001F001F001F001F001F001F6F
:105D3C00001F001F001F001F001F001F001F001E60
:105D4C00001E001E001E001E001E001E001E001E57
:105D5C00001E001E001E001E001E001E001E001E47
:105D6C00001E001E001E001E001E001E001E001E37
:105D7C00001E001E001E001E001E001E001E001E27
:105D8C00001E001E001D001D001D001D001D001D1D
:105D9C00001D001D001D001D001D001D001D001D0F
:105DAC00001D001D001D001D001D001D001D001DFF
:105DBC00001D001D001D001D001D001D001D001DEF
:105DCC00001D001D001D001D001C001C001C001CE3
:105DDC00001C001C001C001C001C001C001C001CD7
:105DEC00001C001C001C001C001C001C001C001CC7
:105DFC00001C001C001C001C001C001C001C001CB7
:105E0C00001C001C001C001C001C001C001B001BA8
:105E1C00001B001B001B001B001B001B001B001B9E
:105E2C00001B001B001B001B001B001B001B001B8E
:105E3C00001B001B001B001B001B001B001B001B7E
:105E4C00001B001B001B001B001B001B001B001B6E
:105E5C00001A001A001A001A001A001A001A001A66
:105E6C00001A001A001A001A001A001A001A001A56
:105E7C00001A001A001A001A001A001A001A001A46
:105E8C00001A001A001A001A001A001A001A001A36
:105E9C00001A001A0019001900190019001900192C
:105EAC00001900190019001900190019001900191E
:105EBC00001900190019001900190019001900190E
:105ECC0000190019001900190019001900190019FE
:105EDC0000190019001900190018001800180018F2
:105EEC0000180018001800180018001800180018E6
:105EFC0000180018001800180018001800180018D6
:105F0C0000180018001800180018001800180018C5
:105F1C0000180018001800180018001800170017B7
:105F2C0000170017001700170017001700170017AD
:105F3C00001700170017001700170017001700179D
:105F4C00001700170017001700170017001700178D
:105F5C00001700170017001700170017001700177D
:105F6C000016001600160016001600160016001675
:105F7C000016001600160016001600160016001665
:105F8C000016001600160016001600160016001655
:105F9C000016001600160016001600160016001645
:105FAC00001600160015001500150015001500153B
:105FBC00001500150015001500150015001500152D
:105FCC00001500150015001500150015001500151D
:105FDC00001500150015001500150015001500150D
:105FEC000015001500150015001400140014001401
:105FFC0000140014001400140014001400140014F5
:10600C0000140014001400140014001400140014E4
:10601C0000140014001400140014001400140014D4
:10602C0000140014001400140014001400140013C5
:10603C0000130013001300130013001300130013BC
:10604C0000130013001300130013001300130013AC
:10605C00001300130013001300130013001300139C
:10606C00001300130013001300130013001300138C
:10607C00001300130013001300130013001300137C
:10608C00001300130013001300130013001300136C
:10609C00001300130013001300130013001300135C
:1060AC00001300130013001300130013001300134C
:1060BC000013001300130012001200120012001241
:1060CC000012001200120012001200120012001234
:1060DC000012001200120012001200120012001224
:1060EC000012001200120012001200120012001214
:1060FC000012001200120012001200120012001204
:10610C0000120012001200120012001200120012F3
:10611C0000120012001200120012001200120012E3
:10612C0000120012001200120012001200120012D3
:10613C0000120012001200120012001200120011C4
:10614C0000110011001100110011001100110011BB
:10615C0000110011001100110011001100110011AB
:10616C00001100110011001100110011001100119B
:10617C00001100110011001100110011001100118B
:10618C00001100110011001100110011001100117B
:10619C00001100110011001100110011001100116B
:1061AC00001100110011001100110011001100115B
:1061BC00001100110011001100110011001100114B
:1061CC000011001100110010001000100010001040
:1061DC000010001000100010001000100010001033
:1061EC000010001000100010001000100010001023
:1061FC000010001000100010001000100010001013
:10620C000010001000100010001000100010001002
:10621C0000100010001000100010001000100010F2
:10622C0000100010001000100010001000100010E2
:10623C0000100010001000100010001000100010D2
:10624C000010001000100010001000100010000FC3
:10625C00000F000F000F000F000F000F000F000FBA
:10626C00000F000F000F000F000F000F000F000FAA
:10627C00000F000F000F000F000F000F000F000F9A
:10628C00000F000F000F000F000F000F000F000F8A
:10629C00000F000F000F000F000F000F000F000F7A
:1062AC00000F000F000F000F000F000F000F000F6A
:1062BC00000F000F000F000F000F000F000F000F5A
:1062CC00000F000F000F000F000F000F000F000F4A
:1062DC00000F000F000F000F000E000E000E000E3E
:1062EC00000E000E000E000E000E000E000E000E32
:1062FC00000E000E000E000E000E000E000E000E22
:10630C00000E000E000E000E000E000E000E000E11
:10631C00000E000E000E000E000E000E000E000E01
:10632C00000E000E000E000E000E000E000E000EF1
:10633C00000E000E000E000E000E000E000E000EE1
:10634C00000E000E000E000E000E000E000E000ED1
:10635C00000E000E000E000E000E000E000E000EC1
:10636C00000D000D000D000D000D000D000D000DB9
:10637C00000D000D000D000D000D000D000D000DA9
:10638C00000D000D000D000D000D000D000D000D99
:10639C00000D000D000D000D000D000D000D000D89
:1063AC00000D000D000D000D000D000D000D000D79
:1063BC00000D000D000D000D000D000D000D000D69
:1063CC00000D000D000D000D000D000D000D000D59
:1063DC00000D000D000D000D000D000D000D000D49
:1063EC00000D000D000D000D000C000C000C000C3D
:1063FC00000C000C000C000C000C000C000C000C31
:10640C00000C000C000C000C000C000C000C000C20
:10641C00000C000C000C000C000C000C000C000C10
:10642C00000C000C000C000C000C000C000C000C00
:10643C00000C000C000C000C000C000C000C000CF0
:10644C00000C000C000C000C000C000C000C000CE0
:10645C00000C000C000C000C000C000C000C000CD0
:10646C00000C000C000C000C000C000C000C000CC0
:10647C00000B000B000B000B000B000B000B000BB8
:10648C00000B000B000B000B000B000B000B000BA8
:10649C00000B000B000B000B000B000B000B000B98
:1064AC00000B000B000B000B000B000B000B000B88
:1064BC00000B000B000B000B000B000B000B000B78
:1064CC00000B000B000B000B000B000B000B000B68
:1064DC00000B000B000B000B000B000B000B000B58
:1064EC00000B000B000B000B000B000B000B000B48
:1064FC00000B000B000B000B000A000A000A000A3C
:10650C00000A000A000A000A000A000A000A000A2F
:10651C00000A000A000A000A000A000A000A000A1F
:10652C00000A000A000A000A000A000A000A000A0F
:10653C00000A000A000A000A000A000A000A000AFF
:10654C00000A000A000A000A000A000A000A000AEF
:10655C00000A000A000A000A000A000A000A000ADF
:10656C00000A000A000A000A000A000A000A000ACF
:10657C00000A000A000A000A000A000A000A000ABF
:10658C00000A0009000900090009000900090009B6
:10659C0000090009000900090009000900090009A7
:1065AC000009000900090009000900090009000997
:1065BC000009000900090009000900090009000987
:1065CC000009000900090009000900090009000977
:1065DC000009000900090009000900090009000967
:1065EC000009000900090009000900090009000957
:1065FC000009000900090009000900090009000947
:10660C000009000900090009000900090009000936
:10661C000009000900090009000900090009000926
:10662C000009000900090009000900090009000916
:10663C000009000900090009000900090009000906
:10664C0000090009000900090009000900090009F6
:10665C0000090009000900090009000900090009E6
:10666C0000090009000900090009000900090009D6
:10667C0000090009000900090009000900090009C6
:10668C0000090009000900090009000900090009B6
:10669C0000090008000800080008000800080008AD
:1066AC00000800080008000800080008000800089E
:1066BC00000800080008000800080008000800088E
:1066CC00000800080008000800080008000800087E
:1066DC00000800080008000800080008000800086E
:1066EC00000800080008000800080008000800085E
:1066FC00000800080008000800080008000800084E
:10670C00000800080008000800080008000800083D
:10671C00000800080008000800080008000800082D
:10672C00000800080008000800080008000800081D
:10673C00000800080008000800080008000800080D
:10674C0000080008000800080008000800080008FD
:10675C0000080008000800080008000800080008ED
:10676C0000080008000800080008000800080008DD
:10677C0000080008000800080008000800080008CD
:10678C0000080008000800080008000800080008BD
:10679C0000080008000800080008000800080008AD
:1067AC0000080007000700070007000700070007A4
:1067BC000007000700070007000700070007000795
:1067CC000007000700070007000700070007000785
:1067DC000007000700070007000700070007000775
:1067EC000007000700070007000700070007000765
:1067FC000007000700070007000700070007000755
:10680C000007000700070007000700070007000744
:10681C000007000700070007000700070007000734
:10682C000007000700070007000700070007000724
:10683C000007000700070007000700070007000714
:10684C000007000700070007000700070007000704
:10685C0000070007000700070007000700070007F4
:10686C0000070007000700070007000700070007E4
:10687C0000070007000700070007000700070007D4
:10688C0000070007000700070007000700070007C4
:10689C0000070007000700070007000700070007B4
:1068AC0000070007000700070007000700070007A4
:1068BC00000700070006000600060006000600069A
:1068CC00000600060006000600060006000600068C
:1068DC00000600060006000600060006000600067C
:1068EC00000600060006000600060006000600066C
:1068FC00000600060006000600060006000600065C
:10690C00000600060006000600060006000600064B
:10691C00000600060006000600060006000600063B
:10692C00000600060006000600060006000600062B
:10693C00000600060006000600060006000600061B
:10694C00000600060006000600060006000600060B
:10695C0000060006000600060006000600060006FB
:10696C0000060006000600060006000600060006EB
:10697C0000060006000600060006000600060006DB
:10698C0000060006000600060006000600060006CB
:10699C0000060006000600060006000600060006BB
:1069AC0000060006000600060006000600060006AB
:1069BC00000600060006000600060006000600069B
:1069CC000006000600050005000500050005000591
:1069DC000005000500050005000500050005000583
:1069EC000005000500050005000500050005000573
:1069FC000005000500050005000500050005000563
:106A0C000005000500050005000500050005000552
:106A1C000005000500050005000500050005000542
:106A2C000005000500050005000500050005000532
:106A3C000005000500050005000500050005000522
:106A4C000005000500050005000500050005000512
:106A5C000005000500050005000500050005000502
:106A6C0000050005000500050005000500050005F2
:106A7C0000050005000500050005000500050005E2
:106A8C0000050005000500050005000500050005D2
:106A9C0000050005000500050005000500050005C2
:106AAC0000050005000500050005000500050005B2
:106ABC0000050005000500050005000500050005A2
:106ACC000005000500050005000500050005000592
:106ADC000005000500050004000400040004000487
:106AEC00000400040004000400040004000400047A
:106AFC00000400040004000400040004000400046A
:106B0C000004000400040004000400040004000459
:106B1C000004000400040004000400040004000449
:106B2C000004000400040004000400040004000439
:106B3C000004000400040004000400040004000429
:106B4C000004000400040004000400040004000419
:106B5C000004000400040004000400040004000409
:106B6C0000040004000400040004000400040004F9
:106B7C0000040004000400040004000400040004E9
:106B8C0000040004000400040004000400040004D9
:106B9C0000040004000400040004000400040004C9
:106BAC0000040004000400040004000400040004B9
:106BBC0000040004000400040004000400040004A9
:106BCC000004000400040004000400040004000499
:106BDC000004000400040004000400040004000489
:106BEC000004000400040004000400040004000479
:106BFC000004000400040004000400040004000469
:106C0C000004000400040004000400040004000458
:106C1C000004000400040004000400040004000448
:106C2C00000400040004000400040003000300033B
:106C3C000003000300030003000300030003000330
:106C4C000003000300030003000300030003000320
:106C5C000003000300030003000300030003000310
:106C6C000003000300030003000300030003000300
:106EDC00000200020001000100010001000100019C
:106EEC00000100010001000100010001000100018E
:106EFC00000100010001000100010001000100017E
:106F0C00000100010001000100010001000100016D
:106F1C00000100010001000100010001000100015D
:106F2C00000100010001000100010001000100014D
:106F3C00000100010001000100010001000100013D
:106F4C00000100010001000100010001000100012D
:106F5C00000100010001000100010001000100011D
:106F6C00000100010001000100010001000100010D
:106F7C0000010001000100010001000100010001FD
:106F8C0000010001000100010001000100010001ED
:106F9C0000010001000100010001000100010001DD
:106FAC0000010001000100010001000100010001CD
:106FBC0000010001000100010001000100010001BD
:106FCC0000010001000100010001000100010001AD
:106FDC00000100010001000100010001000100019D
:106FEC00000100010001000100010001000100018D
:106FFC00000100010001000100010001000100017D
:10700C00000100010001000100010001000100016C
:10701C00000100010001000100010001000100015C
:10702C00000100010001000100010001000100014C
:0D81BE004604AF0000000000004104AE00C8
:1081DE00E4900603F0900603E0FFD39402400302FE
:1081EE0082EBEF25E0246BF582E43404F583E0FCAA
:1081FE00A3E0FDE41242457B007AC0793F78441239
:10820E0041A390060412450E900603E025E024914A
:10821E00F582E43404F583E0FCA3E0FDE41242456C
:10822E00900604E0F8A3E0F9A3E0FAA3E0FB124005
:10823E009A12427E900608EEF0A3EFF0900603E04D
:10824E00FF7E00127F6F900603E0FD25E024AFF560
:10825E0082E43404F583E0FAA3E0D39FEA9E406102
:10826E00EDFF7E00127F6F900603E025E024AFF550
:10827E0082E43404F583E0FCA3E0C39FFFEC9EFE92
:10828E00C3900609E09F900608E09E5047900603B3
:10829E00E0FF25E024AFF582E43404F583C083C00B
:1082AE0082E0FCA3E0FDC004C0057E00127F6FC318
:1082BE00D0E09FFFD0E09ED082D083F0A3EFF0807D
:1082CE0013900603E025E024AFF582E43404F58331
:0D82DE00E4F0A3F0900603E004F00281E359
:0182EB002270
:1072B100E490061CF0A3F07D077C0090061DE025FC
:1072C100E0FF90061CE033FE9004AF75F006ED126E
:1072D100454BEC75F006A42583F583E5822FF582F5
:1072E100E5833EF583E0FAA3E0FB9004B575F00673
:1072F100ED12454BEC75F006A42583F583E5822F4D
:10730100F582E5833EF583EAF0A3EBF0ED1D700114
:107311001CED4C70A690061DE025E0FF90061CE0D8
:1073210033FE746B2FF58274043EF583E0FCA3E019
:10733100FDE41242457B007AC0793F78441241A3B3
:1073410090061E12450E90061DE025E0FF90061CDA
:10735100E033FE74912FF58274043EF583E0FCA3C3
:10736100E0FDE412424590061EE0F8A3E0F9A3E037
:10737100FAA3E0FB12409A12427EAD07AC069006DA
:107381001CE0FAA3E0FB25E0FFEA33FE74B52FF51C
:107391008274043EF583ECF0A3EDF074B52FF58211
:1073A10074043EF583E0FEA3E0D394FFEE940F4016
:1073B10018EB25E0FFEA33FE74B52FF58274043E25
:1073C100F583740FF0A374FFF090061CE0FEA3E0B8
:1073D100FF128AE3AD07AC0690061DE025E0FF90A1
:1073E100061CE033FE74AF2FF58274043EF583E092
:1073F100FAA3E0C39DEA9C500F74AF2FF582740489
:107401003EF583ECF0A3EDF09004AEE004F06402ED
:1074110060030274BB127F67AC06AD0790061DE0E6
:1074210025E0FF90061CE033FE74AF2FF582740453
:107431003EF583E0FEA3E0D39DEE9C4078127F678A
:10744100AC06AD0790061DE025E0FF90061CE03379
:10745100FE74AF2FF58274043EF583E0FAA3E0C316
:107461009DFDEA9CFC74B52FF58274043EF583E022
:10747100FEA3E0C39DEE9C503C90061CE0FCA3E003
:10748100FD25E0FFEC33FE74AF2FF58274043EF569
:1074910083C083C082E0FEA3E0FFC006C007AF0542
:1074A100AE04127F6FC3D0E09FFFD0E09ED082D0A8
:1074B10083F0A3EFF0E49004AEF090061DE004F039
:1074C100700690061CE004F0D390061DE094029033
:0C74D100061CE06480948050030272B836
:0174DD00228C
:087F670090061CE0FEA3E0FF00
:047F6F00AB07AA06AC
:107F7300EB25E0FFEA33FE74AF2FF58274043EF580
:107F830083E0FEA3E0D39466EE94064036EB25E04F
:107F9300FFEA33FE74652FF58274043EF583A3E094
:107FA30025E0FF0582D5820215831582E033FE7436
:107FB3003C2FF58274503EF583E493FC740193FDEA
:107FC3000280B4EB25E0FFEA33FE74AF2FF5827431
:107FD300043EF583E0FEA3E0D39433EE94034039EB
:107FE300EB25E0FFEA33FE74652FF58274043EF55A
:107FF30083A3E025E0FF0582D5820215831582E085
:1080030033FE743C2FF58274503EF583E493C3131F
:10801300FC74019313FD0280B4EB25E0FFEA33FE09
:1080230074AF2FF58274043EF583E0FEA3E0D3948E
:1080330099EE9401403DEB25E0FFEA33FE74652F92
:10804300F58274043EF583A3E025E0FF0582D58223
:108053000215831582E033FE743C2FF58274503E83
:10806300F583E493FE7401937802CEC313CE13D841
:10807300F9803BEB25E0FFEA33FE74652FF582744C
:10808300043EF583A3E025E0FF0582D58202158334
:108093001582E033FE743C2FF58274503EF583E481
:1080A30093FE7401937803CEC313CE13D8F9FDACBA
:0E80B30006ED4C7005FE7F018004AE04AF05A3
:0180C100229C
:10913100D3EF9DEC6480F8EE648098400122AE0488
:03914100AF052255
:108C9400E4FDFCE4FBFAEB25E0FFEA33FE9004B5C7
:108CA40075F006ED12454BEC75F006A42583F583AB
:108CB400E5822FF582E5833EF583E4F0A3F00BBB58
:108CC40000010AEB64034A70CD0DBD00010CED6494
:048CD400084C70BF19
:018CD8002279
:088AE30090063EEEF0A3EFF057
:108AEB00E4A3F0A3F0FBFA90063FE025E0FF90062D
:108AFB003EE033FE9004B575F006EB12454BEA757C
:108B0B00F006A42583F583E5822FF582E5833EF5F8
:108B1B0083E0FCA3E0FD900640E0FEA3E0FF129192
:108B2B0031900640EEF0A3EFF00BBB00010AEB64B3
:0C8B3B00084A70B3900640E0FEA3E0FF83
:018B4700220B
:1081CB0046059400000000000046059A00000000E0
:0281DB000000A2
:1074DE00E4FDFC74232DF58274053CF583E06042D7
:1074EE00ED25E0FFEC33FE74972FF58274043EF524
:1074FE0083E0FAA3E0D39400EA940440028058EDAE
:10750E0025E0FFEC33FE74AF2FF58274043EF58355
:10751E00E0FAA3E0D394FFEA940740030275AF02AA
:10752E0075F0ED25E0FFEC33FE74AF2FF582740499
:10753E003EF583E0FAA3E0D394FFEA9407402B7460
:10754E009A2FF58274053EF583E0FEA3E04E701A85
:10755E00ED25E0FFEC33FE749A2FF58274053EF5AF
:10756E0083E4F0A37402F0027605ED25E0FFEC3320
:10757E00FE74AF2FF58274043EF583E0FAA3E0C3E8
:10758E0094FFEA9407402B749A2FF58274053EF50A
:10759E0083E0FEA3E064024E7018ED25E0FFEC33AD
:1075AE00FE749A2FF58274053EF583E4F0A304F081
:1075BE008045ED25E0FFEC33FE74AF2FF5827404A9
:1075CE003EF583E0FAA3E0C394FFEA9407502874D3
:1075DE009A2FF58274053EF583E0FEA3E064014E1A
:1075EE007015ED25E0FFEC33FE749A2FF5827405CD
:1075FE003EF583E4F0A3F0ED25E0FFEC33FE749A44
:10760E002FF58274053EF583E0FAA3E0FB64024A8F
:10761E00700E74942FF58274053EF583740F8019E5
:10762E00EB64014A701AED25E0FFEC33FE74942FE3
:10763E00F58274053EF5837407F0A374FFF080267F
:10764E00ED25E0FFEC33FE749A2FF58274053EF5BE
:10765E0083E0FAA3E04A700E74942FF58274053E0F
:10766E00F583E4F0A3F00DBD00010CED64034C6056
:04767E00030274E1AE
:0176820022E5
:03000000024000BB
:03000300025003A5
:03000B000250069A
:030013000250098F
:03001B0002500C84
:0300230002500F79
:03002B000250126E
:0300330002501563
:03003B0002501858
:0300430002501B4D
:03004B0002501E42
:0300530002502137
:03005B000250242C
:0300630002502721
:03006B0002502A16
:0300730002502D0B
:03007B0002503000
:03008300025033F5
:03008B00025036EA
:03009300025039DF
:03009B0002503CD4
:0300A30002503FC9
:10400000787FE4F6D8FD9000007F007E20E4F0A3E6
:0A401000DFFCDEFA75812202405544
:10409A00EC4D6011E8497017ED33EC3304600DE420
:1040AA00FCFFFEFD22E933E8330470F80242EA120B
:1040BA0042B558046009E4CC24815006285009020C
:1040CA0042F42840030242F1C0E0EB4A7044B9804E
:1040DA0006D0E0FB0242E0EF4E701CBD8008EBFF09
:1040EA00EAFEE9FD80EBE98DF0A4FEE5F0024183EA
:1040FA00E9CDF9EAFEEBFFEF89F0A4FCE5F0CE8901
:10410A00F0A42EFFE435F0CD89F0A42DFEE435F0BD
:10411A008067EF4E7005BD80D780C3EF8BF0A4ACEB
:10412A00F0EE8BF0A42CFCE435F0F8EF8AF0A42C26
:10413A00E5F038FCE433CB8DF0A42CFCE5F03BF839
:10414A00EE8AF0A42CFCE5F038F8E433CF89F0A429
:10415A002CFCE5F038CF3400CE89F0A42FFFE5F02F
:10416A003EFEE433C98DF0A42EFEE5F039CD8AF087
:10417A00A42FFFE5F03EFEE43DFD33D0E0FB5007FF
:10418A000BBB000F0242F4EC2CFCEF33FFEE33FEC4
:06419A00ED33FD0242CCF2
:1041A0000242F4EC5D046005E8590470030242EA3F
:1041B0001242B5580460F6EC4860F2EC7004FDFE63
:1041C000FF22C860DB2481C85009C39860025006F2
:1041D0000242F19850CAF582E9294B4A7005AB8238
:1041E0000242E075F0007C1A7880C3EF9BEE9AEDF6
:1041F00099400DC3EF9BFFEE9AFEED99FDE842F06A
:10420000DC23ACF0D0E0FFD0E0FED0E0FDAB8220BC
:10421000E7101BEB60BAEC2CFCEF33FFEE33FEED46
:1042200033FD0242CCE803F830E705C0F075F0003A
:10423000EF2FFFEE33FEED33FD40B830E7C280AA2A
:1042400075F020800E75F010800575F0087D007EF9
:10425000007F003392D530D5031244EAEC3340108E
:10426000EF33FFEE33FEED33FDEC33FCD5F0ED2202
:0E427000E5F0247EA2D513CC92E7CDCEFF223E
:10427E00EDD2E7CD33EC3392D524814006E4FFFE38
:10428E00FDFC22FCE4CFCECDCC24E0501174FF8097
:10429E00EDC3CC13CCCD13CDCE13CECF13CF047034
:0742AE00F030D5DE0244EA06
:1042B500E9D2E7C933E833F892D5EDD2E7CD33EC4F
:0742C50033FC5002B2D522C8
:1042CC00EC30E7100FBF000C0EBE00080DBD000453
:1042DC000BEB6014A2D5EB13FCED92E7FD2274FFFF
:1042EC00FCFDFEFF22E480F8A2D574FF13FC7D8058
:0342FC00E480EF6C
:10401A0002703CE493A3F8E493A34003F68001F210
:10402A0008DFF48029E493A3F85407240CC8C333A7
:10403A00C4540F4420C8834004F456800146F6DF76
:10404A00E4800B01020408102040809080C2E47EC4
:10405A00019360BCA3FF543F30E509541FFEE4936B
:10406A00A360010ECF54C025E060A840B8E493A332
:10407A00FAE493A3F8E493A3C8C582C8CAC583CA5D
:10408A00F0A3C8C582C8CAC583CADFE9DEE780BE15
:0181DD0000A1
:1042FF00E709F608DFFA8046E709F208DFFA803EA1
:10430F0088828C83E709F0A3DFFA8032E309F6088D
:10431F00DFFA8078E309F208DFFA807088828C83F5
:10432F00E309F0A3DFFA806489828A83E0A3F608A9
:10433F00DFFA805889828A83E0A3F208DFFA804C83
:10434F0080D280FA80C680D4806980F2803380105A
:10435F0080A680EA809A80A880DA80E280CA8033C3
:10436F0089828A83ECFAE493A3C8C582C8CCC5833B
:10437F00CCF0A3C8C582C8CCC583CCDFE9DEE7800B
:10438F000D89828A83E493A3F608DFF9ECFAA9F08A
:10439F00EDFB2289828A83ECFAE0A3C8C582C8CCE0
:1043AF00C583CCF0A3C8C582C8CCC583CCDFEADEF9
:1043BF00E880DB89828A83E493A3F208DFF980CC5B
:1043CF0088F0EF60010E4E60C388F0ED2402B40454
:1043DF000050B9F582EB2402B4040050AF232345FB
:0643EF00822390434F738E
:1043F500BB010689828A83E0225002E722BBFE02C6
:09440500E32289828A83E49322F8
:10440E00BB010CE58229F582E5833AF583E0225063
:10441E0006E92582F8E622BBFE06E92582F8E222AD
:0D442E00E58229F582E5833AF583E49322C7
:10443B00BB010689828A83F0225002F722BBFE0160
:02444B00F3225A
:10444D00F8BB010DE58229F582E5833AF583E8F0A5
:10445D00225006E92582C8F622BBFE05E92582C851
:02446D00F22239
:10446F00C5F0F8A3E028F0C5F0F8E58215827002D8
:06447F001583E038F02275
:10448500A3F8E0C5F025F0F0E582158270021583EA
:06449500E0C838F0E82247
:10449B00E88FF0A4CC8BF0A42CFCE98EF0A42CFCC0
:1044AB008AF0EDA42CFCEA8EF0A4CDA8F08BF0A43E
:1044BB002DCC3825F0FDE98FF0A42CCD35F0FCEB9D
:1044CB008EF0A4FEA9F0EB8FF0A4CFC5F02ECD3962
:0F44DB00FEE43CFCEAA42DCE35F0FDE43CFC22CF
:108D1D00C2D5E830E70FB2D5E4C39BFBE49AFAE481
:108D2D0099F9E498F8EC30E717B2D5128D53124645
:108D3D0016E4C39BFBE49AFAE499F9E498F88003EE
:108D4D0012461630D50DE4C39FFFE49EFEE49DFD53
:048D5D00E49CFC2274
:0E44EA00C3E49FFFE49EFEE49DFDE49CFC22E3
:1044F800EB9FF5F0EA9E42F0E99D42F0EC6480C83B
:0645080064809845F022DA
:0C450E00ECF0A3EDF0A3EEF0A3EFF02220
:10451A00A8828583F0D083D08212453112453112A8
:10452A004531124531E473E493A3C583C5F0C583CD
:10453A00C8C582C8F0A3C583C5F0C583C8C582C8EB
:01454A00224E
:0C454B00A42582F582E5F03583F583227B
:10455700D083D082F8E4937012740193700DA3A3F3
:1045670093F8740193F5828883E473740293686007
:06457700EFA3A3A380DF07
:10457D00E50D2582F582E50C3583F583B50C0485B3
:10458D00820D2210AF0685820DF50C2285820DF568
:04459D000CD2AF226B
:0D45A100E50D2582F582E50C3583F58322BA
:1045AE00EF4E6012EF60010EEDBB010B89828A8324
:1045BE00F0A3DFFCDEFA2289F05007F709DFFCA931
:0C45CE00F022BBFEFCF309DFFCA9F02288
:1045DA0075F008758200EF2FFFEE33FECD33CDCC98
:1045EA0033CCC58233C5829BED9AEC99E58298401B
:1045FA000CF582EE9BFEED9AFDEC99FC0FD5F0D6F8
:10460A00E4CEFBE4CDFAE4CCF9A88222B800C1B921
:10461A000059BA002DEC8BF084CFCECDFCE5F0CB5F
:10462A00F97818EF2FFFEE33FEED33FDEC33FCEB98
:10463A0033FB10D703994004EB99FB0FD8E5E4F953
:10464A00FA227818EF2FFFEE33FEED33FDEC33FC40
:10465A00C933C910D7059BE99A4007EC9BFCE99A34
:10466A00F90FD8E0E4C9FAE4CCFB2275F010EF2F79
:10467A00FFEE33FEED33FDCC33CCC833C810D70779
:10468A009BEC9AE899400AED9BFDEC9AFCE899F8B4
:0E469A000FD5F0DAE4CDFBE4CCFAE4C8F92247
:00000001FF
